:0A28F4004216AF00004216B20000C9
:102DF3007811E604540FFF780DE622780EE60454AA
:062E030003FF780CE6223B
:102E1F00780DE6FF7811666007EF04540F780DF612
:012E2F002280
:0A2E5200122DF36F60047811A6073B
:012E5C002253
:092E7300122DF3B50702C322D3AE
:012E7C002233
:102E3000780CE6FF780E666007EF045403780CF612
:012E4000226F
:0A2E5D00122DFE6F6004780EA60728
:012E67002248
:092E7D00122DFEB50702C322D399
:012E86002229
:10032900E4781BF6D2B6C2B7782576C8122EB3C2C6
:10033900A6122EAC122E689003127401F090020CD2
:10034900F0900106F0900000F090072AF090062442
:10035900F090051EF0900418F0900B42F0900A3CC2
:10036900F0900936F0900830F0900F5AF0900E5442
:10037900F0900D4EF0900C48F0E4780FF608F678FE
:1003890013F6780BF618F67808F67812F618F67858
:100399000DF608F6780CF6122EA39016AFE0FEA320
:1003A900E0FF9016B2E06E7003A3E06F600A90164A
:1003B900B2EEF0A3EFF0B2B67816E66014781B0639
:1003C900E6D394024007A2B7B392B7E4F6E47816ED
:1003D900F6120094780DE6B41000400302046D9003
:1003E90003EFF828287302041F02042402042902D7
:1003F900042E02043302043802043D0204420204BA
:100409004702044C02045102045602045B020460D0
:1004190002046502046A12282C804912289080443B
:1004290012228A803F1222F1803A12235880351213
:1004390023BF8030122426802B12248D802612247B
:10044900F4802112255B801C1225C28017122629EF
:100459008012122690800D1226F7800812275E80DE
:10046900031227C5780EE614601314601614601978
:10047900240360030203A01204980203A012089A3D
:0F0489000203A01205EE0203A01207440203A013
:0C28FE0001210001220002230000C18320
:0D001600D2A0D37815E6940018E6940022DD
:0300030002000EEA
:03000E00C20332F8
:03001300022DC1FA
:102DC100C0E0C083C0829016B0E004F07006901697
:0B2DD100AFE004F0D082D083D0E032ED
:102D8400C200C201C203D288D2A8D28AD2AAD20275
:102D9400120B3AEF4E6009C202120B3AEF4E70F773
:012DA400220C
:092E9100D2037F017E00022CF146
:032EBA00C28022B1
:032EBD00D280229E
:040026007F8A7E024D
:10002A007590FF7814A60608A6077590FF00D2A25D
:10003A00D2A1C2A000AF901200164004EF20E0EA5D
:10004A00A203B34004EF30E003D38001C39204302B
:10005A0004037FFF22C2A2D2A1C2A000AF90D2A005
:01006A002273
:10292F007814760208768A7590FF00D2A2D2A1C2DF
:10293F00A000AE901200164004EE20E0EAA203B30E
:10294F004004EE30E003D38001C3920420040B8FC8
:0A295F0090C2A2C2A1C2A000D2A043
:01296900224B
:01000A0022D3
:100B3A00E49016A4F07821F608F6C2B612000A125A
:100B4A002EBA7F0AFE122CF1122EBDA2B6B392B6AD
:100B5A0012000A7F0A120C37A2B6B392B67F641249
:100B6A000C377F2C7E01122CF1A2B6B392B612007A
:100B7A000AD2B67F5A12292F300403020C27E4FF47
:100B8A0012292F3004028069120026EF64076003DD
:100B9A00020C27E4FF12292F3004028054E4FF12CA
:100BAA00292F300402804A7F587E0212002AEF64FD
:100BBA000160028068120026EF64016002805E1202
:100BCA000026EF6450600280547F0112292F3004FE
:100BDA00037E00227F0112292F3004037E00227F28
:100BEA006012292F3004028034E4FF12292F3004C6
:100BFA00047E000F227F587E0212002A30040280EF
:100C0A001CEF6021640160028013120026AD0730D8
:100C1A0004028009ED600E1200263004057E007F72
:0C0C2A0001221D80EF78217601E4FEFF1E
:0D0C3600227E00122CF1122E9112000A22D3
:10009400122E7340030203287811E62484F582E4C7
:1000A4003416F583E060030203282003030201B938
:1000B4007821E66401705478230806E61870010676
:1000C4008606D39410EE940040277F5A12292F30CD
:1000D40004030201B9E4FF12292F3004030201B919
:1000E400120026EF640760030201B9E47823F608DE
:1000F400F6E4FF12292F3004030201B9E4FF1229A8
:100104002F3004030201B9782176037811E6B41084
:100114000040030201A3900121F828287302015131
:1001240002015602015B02016002016502016A02DA
:10013400016F02017402017902017E02018302014E
:100144008802018D02019202019702019C120D475F
:100154008049120E478044120F47803F1210478097
:100164003A12114780351212478030121347802B00
:1001740012144780261215478021121647801C123C
:10018400174780171218478012121947800D121A48
:10019400478008121B478003121C47781CA6077867
:1001A4001CE60470030203131460030202CA7822DB
:1001B40076020202CAC202120B3AEF4E70F77811AD
:1001C400E6FFB4100040030202BA9001D5F82828D3
:1001D4007302020502021102021D02022902023503
:1001E40002024002024B02025602026102026C0247
:1001F400027702028202028D0202980202A3020224
:10020400AE9000047450F09000020202B790010A0C
:100214007450F09001080202B79002107450F090EC
:10022400020E0202B79003167450F09003140202F7
:10023400B790041C7450F090041A807790052274CF
:1002440050F0900520806C9006287450F09006269B
:10025400806190072E7450F090072C8056900628E9
:100264007450F0900832804B90072E7450F090092F
:10027400388040900A407450F0900A3E8035900BCC
:10028400467450F0900B44802A900C4C7450F090BB
:100294000C4A801F900D527450F0900D50801490B1
:1002A4000E587450F0900E568009900F5E7450F002
:1002B400900F5C7401F074842FF582E43416F58396
:1002C4007401F0122E5278217601780CE6FF248016
:1002D400F582E43416F583E0604A7822E66401602E
:1002E40043EF14601214601714601C24037020126E
:1002F4001E45501B0201B9121EF350130201B9121C
:100304001FA1500B0201B912204F50030201B9780A
:10031400217603E4FF12292F3004030201B9E478A3
:0403240023F608F6BE
:0103280022B2
:0A2E87009016A5F0A3EFF0D2A922E7
:102CF100C2A97814A60608A607EE122E879016A57B
:102D0100E07002A3E06011C2A97814E6FF08E6CFE3
:082D1100122E87122EA380E5AB
:012D19002297
:072EAC009016B17402F02240
:03000B0002219A35
:10219A00C0E0C0F0C083C082C0D075D000C000C00B
:1021AA0001C002C003C004C005C006C007C28C75C6
:1021BA008CF4758A00D28C7825E6FF600675A61E17
:1021CA0075A6E17815E61846600708E61618700144
:1021DA0016781716E6701E760A0876010876010840
:1021EA0016E67011760A78167601EF6005782516DC
:1021FA008003120006D007D006D005D004D003D041
:10220A0002D001D000D0D0D082D083D0F0D0E0323A
:102E09007817760A781A760A438901758CF4E4F5FD
:062E19008AD2A9D28C222E
:0B2E6800122E09122D3FD2AF022D8464
:10006B0075878075985075CBFF75CAF675C834D2F5
:04007B00BCD2AC2225
:102DDC00758780759850539BEC439B0E759AF64300
:072DEC009B10D2BCD2AC2207
:102D3F007E147F7A122E9A7E157F7D122E9AC205EF
:102D4F009016B1E0FFB4010302006BEFB40203125F
:032D5F002DDC2246
:102DA500A2AF9200C2AF20050E7E157F7D122E4187
:0B2DB500EF6004D299D205A20092AF9B
:012DC00022F0
:0300230002221A9C
:10221A00C0E0C083C082C0D075D000C005C006C06F
:01222A0007AC
:10222B00309825AF9990147AE0FE04FDA3E06D6021
:10223B0013747D2EF582E43414F583EFF0AF059023
:10224B00147AEFF0C298802830992590157EE0FF24
:10225B0090157DE06F601574802FF582E43415F5D1
:10226B0083E0F59990157EE004F08002C205C299D7
:0F227B00D007D006D005D0D0D082D083D0E032AB
:1029A300EEF0A3EFF0A3EBF0A3EAF0A3E9F0E42247
:1029B300E0FEA3E0FFA3E0FBA3E0FAA3E0F922A378
:1029C300A3A32582F582E43583F583228F828E8348
:0329D300A3E0225C
:102D62008F828E83E004F9A3E0B501037F00228FF6
:102D7200828E83E01229C2EDF08F828E83E9F07F8A
:012D8200014F
:012D8300222D
:092E9A008F828E83E4F0A3F02284
:0329D6009016A4B4
:1029D9001229A3FC9016A9E0FFECC39F501D901685
:1029E900A41229B3120AE3FD122D62EF600D0C90B7
:0D29F90016A7E475F001120B0E80D9AF0493
:012A060022AD
:03296A009016A81C
:10296D001229A39016AEF09016ADE0FFA3E0C39F21
:10297D00501E9016A81229B3122D1AEF6012901640
:10298D00AEE004F09016ABE475F001120B0E80D79B
:05299D009016AEE0FF02
:0129A2002212
:102D1A001229CFFD8F828E83E0B505037F00221230
:102D2A0029CF8F828E831229C2E0120AFC1229CF80
:052D3A0004F07F0122FE
:102E41008F828E83E0FFA3E0B507037F00227F011D
:012E5100225E
:030000000220FDDE
:1020FD0078FFE4F6D8FD538EFD9000007FFF7E1F24
:0D210D00E4F0A3DFFCDEFA75812502215508
:101D4700E6FF7E0078807C157D017B01120ABDE4E9
:101D570090157EF0227808E6F0A3E0FFF4A3F01FC9
:101D6700A3E0FEAD0722AF90D2A0D37815E694008A
:101D770018E69400227E157F7D7B01E69016A9F078
:101D87002278130678107607E4780AF622E6FF7EB3
:101D97000078807C157D017B01227590FF78147691
:101DA7000208768A22A60790157DE0FFA3E06F223E
:101DB7007E157F7D7B01E69016A9F022E4F6780A6E
:101DC70006E6D3940A227E157F7D7B01E69016A94D
:101DD700F022D3ED94007480948122F583E590F08E
:101DE700D2A00622F583EEF0EF2406FF227E157FB0
:101DF7007D7B01E69016A9F0227E157F7D7B01E6AB
:101E07009016A9F022D2A2D2A1C2A022C2A2D2A128
:101E1700C2A0227813E6D39405227E157F7D7B012D
:101E2700E69016A9F0227E157F7D7B01E69016A924
:0E1E3700F0227E157F7D7B01E69016A9F02239
:100D47007F58120E3D20040E781FE6FE70037F01C8
:100D570022EE6401601FC202120B3AEF4E70F79049
:100D670000047450F09000027401F0901684F012A1
:100D77002E527F01227F8A7E0212002A781EA60742
:100D87002004D37F8A120E3D2004CB781FE6FEB4E1
:100D9700C0037F0022781EE6FD70037F0122121D2B
:100DA700D950B3900004EEF0781EE616900002F0DA
:100DB700E418F6791DE7C3781E96503C121DA175FD
:100DC70090FF00121E0C00121D6D4004EF20E0EF93
:100DD700A203B34004EF30E003D38001C392043091
:100DE7000403020D5D121E1300781DE62405F5822B
:100DF700E43400121DE280BB9016847401F0122EB9
:100E070052781FE66450702B18E670277822F67F19
:100E17000112292F3004037F01227F0112292F306D
:100E270004037F01227F6012292F3004037F0122F0
:050E37007FFF227F0196
:0B0E3C00227E0212002A781FA6072267
:102C9900900001121D5CEDD3940040101D74052DA8
:102CA900F582E43400F583E02EFE80EAEEF404FEBA
:0B2CB90074052FF582E43400121DEBBF
:012CC40022ED
:10282C00901684E0605D7810E67031122C99781C5B
:10283C00121DAC60107A007900121D7C1229D6781A
:10284C001CA6078010781C7A007900121D47781C92
:10285C00E690157DF0122DA5121D88227818E660E1
:10286C0022121DC3401D121E1A4014E4901684F04F
:10287C00122E1F780806E670027601E47813F6E44F
:03288C007810F6CB
:01288F002226
:100E47007F58120F3D20040E781FE6FE70037F01C6
:100E570022EE6401601FC202120B3AEF4E70F79048
:100E6700010A7450F09001087401F0901685F01291
:100E77002E527F01227F8A7E0212002A781EA60741
:100E87002004D37F8A120F3D2004CB781FE6FEB4DF
:100E9700C0037F0022781EE6FD70037F0122121D2A
:100EA700D950B390010AEEF0781EE616900108F0CB
:100EB700E418F6791DE7C3781E96503C121DA175FC
:100EC70090FF00121E0C00121D6D4004EF20E0EF92
:100ED700A203B34004EF30E003D38001C392043090
:100EE7000403020E5D121E1300781DE6240BF58223
:100EF700E43401121DE280BB9016857401F0122EB6
:100F070052781FE66450702B18E670277822F67F18
:100F17000112292F3004037F01227F0112292F306C
:100F270004037F01227F6012292F3004037F0122EF
:050F37007FFF227F0195
:0B0F3C00227E0212002A781FA6072266
:102CC500900107121D5CEDD3940040101D740B2D6F
:102CD500F582E43401F583E02EFE80EAEEF404FE8D
:0B2CE500740B2FF582E43401121DEB8C
:012CF00022C1
:10289000901685E0605D7810E67031122CC5781CCA
:1028A000121DAC60107A017906121D7C1229D678AF
:1028B0001CA6078010781C7A017906121D47781C27
:1028C000E690157DF0122DA5121D88227818E6607D
:1028D00022121DC3401D121E1A4014E4901685F0EA
:1028E000122E1F780806E670027601E47813F6E4EB
:0328F0007810F667
:0128F30022C2
:100F47007F5812103D20040E781FE6FE70037F01C4
:100F570022EE6401601FC202120B3AEF4E70F79047
:100F670002107450F090020E7401F0901686F01281
:100F77002E527F01227F8A7E0212002A781EA60740
:100F87002004D37F8A12103D2004CB781FE6FEB4DD
:100F9700C0037F0022781EE6FD70037F0122121D29
:100FA700D950B3900210EEF0781EE61690020EF0BC
:100FB700E418F6791DE7C3781E96503C121DA175FB
:100FC70090FF00121E0C00121D6D4004EF20E0EF91
:100FD700A203B34004EF30E003D38001C39204308F
:100FE7000403020F5D121E1300781DE62411F5821B
:100FF700E43402121DE280BB9016867401F0122EB3
:1010070052781FE66450702B18E670277822F67F17
:101017000112292F3004037F01227F0112292F306B
:1010270004037F01227F6012292F3004037F0122EE
:051037007FFF227F0194
:0B103C00227E0212002A781FA6072265
:102A07007808E690020D121D5FEDD3940040101D6B
:102A170074112DF582E43402F583E02EFE80EAEE90
:0E2A2700F404FE74112FF582E43402121DEB4C
:012A3500227E
:10228A00901686E060607810E67034122A07781C8F
:10229A00121DAC60107A02790C121DB71229D67879
:1022AA001CA6078013781C121D947A02790C121D41
:1022BA0053781CE690157DF0122DA5121D88227800
:1022CA0018E66022121DC3401D121E1A4014E49023
:1022DA001686F0122E1F780806E670027601E47858
:0622EA0013F6E47810F683
:0122F00022CB
:101047007F5812113D20040E781FE6FE70037F01C2
:1010570022EE6401601FC202120B3AEF4E70F79046
:1010670003167450F09003147401F0901687F01271
:101077002E527F01227F8A7E0212002A781EA6073F
:101087002004D37F8A12113D2004CB781FE6FEB4DB
:10109700C0037F0022781EE6FD70037F0122121D28
:1010A700D950B3900316EEF0781EE616900314F0AD
:1010B700E418F6791DE7C3781E96503C121DA175FA
:1010C70090FF00121E0C00121D6D4004EF20E0EF90
:1010D700A203B34004EF30E003D38001C39204308E
:1010E700040302105D121E1300781DE62417F58213
:1010F700E43403121DE280BB9016877401F0122EB0
:1011070052781FE66450702B18E670277822F67F16
:101117000112292F3004037F01227F0112292F306A
:1011270004037F01227F6012292F3004037F0122ED
:051137007FFF227F0193
:0B113C00227E0212002A781FA6072264
:102A36007808E6900313121D5FEDD3940040101D35
:102A460074172DF582E43403F583E02EFE80EAEE5A
:0E2A5600F404FE74172FF582E43403121DEB16
:012A6400224F
:1022F100901687E060607810E67034122A36781CF8
:10230100121DAC60107A037912121DB71229D6780A
:102311001CA6078013781C121D947A037912121DD2
:1023210053781CE690157DF0122DA5121D88227898
:1023310018E66022121DC3401D121E1A4014E490BB
:102341001687F0122E1F780806E670027601E478EF
:0623510013F6E47810F61B
:012357002263
:101147007F5812123D20040E781FE6FE70037F01C0
:1011570022EE6401601FC202120B3AEF4E70F79045
:10116700041C7450F090041A7401F0901688F01261
:101177002E527F01227F8A7E0212002A781EA6073E
:101187002004D37F8A12123D2004CB781FE6FEB4D9
:10119700C0037F0022781EE6FD70037F0122121D27
:1011A700D950B390041CEEF0781EE61690041AF09E
:1011B700E418F6791DE7C3781E96503C121DA175F9
:1011C70090FF00121E0C00121D6D4004EF20E0EF8F
:1011D700A203B34004EF30E003D38001C39204308D
:1011E700040302115D121E1300781DE6241DF5820B
:1011F700E43404121DE280BB9016887401F0122EAD
:1012070052781FE66450702B18E670277822F67F15
:101217000112292F3004037F01227F0112292F3069
:1012270004037F01227F6012292F3004037F0122EC
:051237007FFF227F0192
:0B123C00227E0212002A781FA6072263
:102A65007808E6900419121D5FEDD3940040101DFF
:102A7500741D2DF582E43404F583E02EFE80EAEE24
:0E2A8500F404FE741D2FF582E43404121DEBE0
:012A93002220
:10235800901688E060607810E67034122A65781C60
:10236800121DAC60107A047918121DCD1229D67886
:102378001CA6078013781C121D947A047918121D64
:1023880053781CE690157DF0122DA5121D88227831
:1023980018E66022121DC3401D121E1A4014E49054
:1023A8001688F0122E1F780806E670027601E47887
:0623B80013F6E47810F6B4
:0123BE0022FC
:101247007F5812133D20040E781FE6FE70037F01BE
:1012570022EE6401601FC202120B3AEF4E70F79044
:1012670005227450F09005207401F0901689F01251
:101277002E527F01227F8A7E0212002A781EA6073D
:101287002004D37F8A12133D2004CB781FE6FEB4D7
:10129700C0037F0022781EE6FD70037F0122121D26
:1012A700D950B3900522EEF0781EE616900520F08F
:1012B700E418F6791DE7C3781E96503C121DA175F8
:1012C70090FF00121E0C00121D6D4004EF20E0EF8E
:1012D700A203B34004EF30E003D38001C39204308C
:1012E700040302125D121E1300781DE62423F58203
:1012F700E43405121DE280BB9016897401F0122EAA
:1013070052781FE66450702B18E670277822F67F14
:101317000112292F3004037F01227F0112292F3068
:1013270004037F01227F6012292F3004037F0122EB
:051337007FFF227F0191
:0B133C00227E0212002A781FA6072262
:102A94007808E690051F121D5FEDD3940040101DC9
:102AA40074232DF582E43405F583E02EFE80EAEEEE
:0E2AB400F404FE74232FF582E43405121DEBAA
:012AC20022F1
:1023BF00901689E060607810E67034122A94781CC9
:1023CF00121DAC60107A05791E121DCD1229D67818
:1023DF001CA6078013781C121D947A05791E121DF6
:1023EF0053781CE690157DF0122DA5121D882278CA
:1023FF0018E66022121DC3401D121E1A4014E490ED
:10240F001689F0122E1F780806E670027601E4781E
:06241F0013F6E47810F64C
:012425002294
:101347007F5812143D20040E781FE6FE70037F01BC
:1013570022EE6401601FC202120B3AEF4E70F79043
:1013670006287450F09006267401F090168AF01241
:101377002E527F01227F8A7E0212002A781EA6073C
:101387002004D37F8A12143D2004CB781FE6FEB4D5
:10139700C0037F0022781EE6FD70037F0122121D25
:1013A700D950B3900628EEF0781EE616900626F080
:1013B700E418F6791DE7C3781E96503C121DA175F7
:1013C70090FF00121E0C00121D6D4004EF20E0EF8D
:1013D700A203B34004EF30E003D38001C39204308B
:1013E700040302135D121E1300781DE62429F582FB
:1013F700E43406121DE280BB90168A7401F0122EA7
:1014070052781FE66450702B18E670277822F67F13
:101417000112292F3004037F01227F0112292F3067
:1014270004037F01227F6012292F3004037F0122EA
:051437007FFF227F0190
:0B143C00227E0212002A781FA6072261
:102AC3007808E6900625121D5FEDD3940040101D93
:102AD30074292DF582E43406F583E02EFE80EAEEB8
:0E2AE300F404FE74292FF582E43406121DEB74
:012AF10022C2
:1024260090168AE060607810E67034122AC3781C31
:10243600121DAC60107A067924121DF41229D67882
:102446001CA6078013781C121D947A067924121D87
:1024560053781CE690157DF0122DA5121D88227862
:1024660018E66022121DC3401D121E1A4014E49085
:10247600168AF0122E1F780806E670027601E478B6
:0624860013F6E47810F6E5
:01248C00222D
:101447007F5812153D20040E781FE6FE70037F01BA
:1014570022EE6401601FC202120B3AEF4E70F79042
:10146700072E7450F090072C7401F090168BF01231
:101477002E527F01227F8A7E0212002A781EA6073B
:101487002004D37F8A12153D2004CB781FE6FEB4D3
:10149700C0037F0022781EE6FD70037F0122121D24
:1014A700D950B390072EEEF0781EE61690072CF071
:1014B700E418F6791DE7C3781E96503C121DA175F6
:1014C70090FF00121E0C00121D6D4004EF20E0EF8C
:1014D700A203B34004EF30E003D38001C39204308A
:1014E700040302145D121E1300781DE6242FF582F3
:1014F700E43407121DE280BB90168B7401F0122EA4
:1015070052781FE66450702B18E670277822F67F12
:101517000112292F3004037F01227F0112292F3066
:1015270004037F01227F6012292F3004037F0122E9
:051537007FFF227F018F
:0B153C00227E0212002A781FA6072260
:102AF2007808E690072B121D5FEDD3940040101D5D
:102B0200742F2DF582E43407F583E02EFE80EAEE81
:0E2B1200F404FE742F2FF582E43407121DEB3D
:012B20002292
:10248D0090168BE060607810E67034122AF2781C9A
:10249D00121DAC60107A07792A121DF41229D67814
:1024AD001CA6078013781C121D947A07792A121D19
:1024BD0053781CE690157DF0122DA5121D882278FB
:1024CD0018E66022121DC3401D121E1A4014E4901E
:1024DD00168BF0122E1F780806E670027601E4784E
:0624ED0013F6E47810F67E
:0124F30022C6
:101547007F5812163D20040E781FE6FE70037F01B8
:1015570022EE6401601FC202120B3AEF4E70F79041
:1015670008347450F09008327401F090168CF01221
:101577002E527F01227F8A7E0212002A781EA6073A
:101587002004D37F8A12163D2004CB781FE6FEB4D1
:10159700C0037F0022781EE6FD70037F0122121D23
:1015A700D950B3900834EEF0781EE616900832F062
:1015B700E418F6791DE7C3781E96503C121DA175F5
:1015C70090FF00121E0C00121D6D4004EF20E0EF8B
:1015D700A203B34004EF30E003D38001C392043089
:1015E700040302155D121E1300781DE62435F582EB
:1015F700E43408121DE280BB90168C7401F0122EA1
:1016070052781FE66450702B18E670277822F67F11
:101617000112292F3004037F01227F0112292F3065
:1016270004037F01227F6012292F3004037F0122E8
:051637007FFF227F018E
:0B163C00227E0212002A781FA607225F
:102B21007808E6900831121D5FEDD3940040101D26
:102B310074352DF582E43408F583E02EFE80EAEE4B
:0E2B4100F404FE74352FF582E43408121DEB07
:012B4F002263
:1024F40090168CE060607810E67034122B21781C02
:10250400121DAC60107A087930121E001229D67898
:102514001CA6078013781C121D947A087930121DAA
:1025240053781CE690157DF0122DA5121D88227893
:1025340018E66022121DC3401D121E1A4014E490B6
:10254400168CF0122E1F780806E670027601E478E5
:0625540013F6E47810F616
:01255A00225E
:101647007F5812173D20040E781FE6FE70037F01B6
:1016570022EE6401601FC202120B3AEF4E70F79040
:10166700093A7450F09009387401F090168DF01211
:101677002E527F01227F8A7E0212002A781EA60739
:101687002004D37F8A12173D2004CB781FE6FEB4CF
:10169700C0037F0022781EE6FD70037F0122121D22
:1016A700D950B390093AEEF0781EE616900938F053
:1016B700E418F6791DE7C3781E96503C121DA175F4
:1016C70090FF00121E0C00121D6D4004EF20E0EF8A
:1016D700A203B34004EF30E003D38001C392043088
:1016E700040302165D121E1300781DE6243BF582E3
:1016F700E43409121DE280BB90168D7401F0122E9E
:1017070052781FE66450702B18E670277822F67F10
:101717000112292F3004037F01227F0112292F3064
:1017270004037F01227F6012292F3004037F0122E7
:051737007FFF227F018D
:0B173C00227E0212002A781FA607225E
:102B50007808E6900937121D5FEDD3940040101DF0
:102B6000743B2DF582E43409F583E02EFE80EAEE15
:0E2B7000F404FE743B2FF582E43409121DEBD1
:012B7E002234
:10255B0090168DE060607810E67034122B50781C6A
:10256B00121DAC60107A097936121E001229D6782A
:10257B001CA6078013781C121D947A097936121D3C
:10258B0053781CE690157DF0122DA5121D8822782C
:10259B0018E66022121DC3401D121E1A4014E4904F
:1025AB00168DF0122E1F780806E670027601E4787D
:0625BB0013F6E47810F6AF
:0125C10022F7
:101747007F5812183D20040E781FE6FE70037F01B4
:1017570022EE6401601FC202120B3AEF4E70F7903F
:101767000A407450F0900A3E7401F090168EF01201
:101777002E527F01227F8A7E0212002A781EA60738
:101787002004D37F8A12183D2004CB781FE6FEB4CD
:10179700C0037F0022781EE6FD70037F0122121D21
:1017A700D950B3900A40EEF0781EE616900A3EF044
:1017B700E418F6791DE7C3781E96503C121DA175F3
:1017C70090FF00121E0C00121D6D4004EF20E0EF89
:1017D700A203B34004EF30E003D38001C392043087
:1017E700040302175D121E1300781DE62441F582DB
:1017F700E4340A121DE280BB90168E7401F0122E9B
:1018070052781FE66450702B18E670277822F67F0F
:101817000112292F3004037F01227F0112292F3063
:1018270004037F01227F6012292F3004037F0122E6
:051837007FFF227F018C
:0B183C00227E0212002A781FA607225D
:102B7F007808E6900A3D121D5FEDD3940040101DBA
:102B8F0074412DF582E4340AF583E02EFE80EAEEDF
:0E2B9F00F404FE74412FF582E4340A121DEB9B
:012BAD002205
:1025C20090168EE060607810E67034122B7F781CD3
:1025D200121DAC60107A0A793C121E211229D6789B
:1025E2001CA6078013781C121D947A0A793C121DCE
:1025F20053781CE690157DF0122DA5121D882278C5
:1026020018E66022121DC3401D121E1A4014E490E7
:10261200168EF0122E1F780806E670027601E47814
:0626220013F6E47810F647
:01262800228F
:101847007F5812193D20040E781FE6FE70037F01B2
:1018570022EE6401601FC202120B3AEF4E70F7903E
:101867000B467450F0900B447401F090168FF012F1
:101877002E527F01227F8A7E0212002A781EA60737
:101887002004D37F8A12193D2004CB781FE6FEB4CB
:10189700C0037F0022781EE6FD70037F0122121D20
:1018A700D950B3900B46EEF0781EE616900B44F035
:1018B700E418F6791DE7C3781E96503C121DA175F2
:1018C70090FF00121E0C00121D6D4004EF20E0EF88
:1018D700A203B34004EF30E003D38001C392043086
:1018E700040302185D121E1300781DE62447F582D3
:1018F700E4340B121DE280BB90168F7401F0122E98
:1019070052781FE66450702B18E670277822F67F0E
:101917000112292F3004037F01227F0112292F3062
:1019270004037F01227F6012292F3004037F0122E5
:051937007FFF227F018B
:0B193C00227E0212002A781FA607225C
:102BAE007808E6900B43121D5FEDD3940040101D84
:102BBE0074472DF582E4340BF583E02EFE80EAEEA9
:0E2BCE00F404FE74472FF582E4340B121DEB65
:012BDC0022D6
:1026290090168FE060607810E67034122BAE781C3B
:10263900121DAC60107A0B7942121E211229D6782C
:102649001CA6078013781C121D947A0B7942121D5F
:1026590053781CE690157DF0122DA5121D8822785D
:1026690018E66022121DC3401D121E1A4014E49080
:10267900168FF0122E1F780806E670027601E478AC
:0626890013F6E47810F6E0
:01268F002228
:101947007F58121A3D20040E781FE6FE70037F01B0
:1019570022EE6401601FC202120B3AEF4E70F7903D
:101967000C4C7450F0900C4A7401F0901690F012E1
:101977002E527F01227F8A7E0212002A781EA60736
:101987002004D37F8A121A3D2004CB781FE6FEB4C9
:10199700C0037F0022781EE6FD70037F0122121D1F
:1019A700D950B3900C4CEEF0781EE616900C4AF026
:1019B700E418F6791DE7C3781E96503C121DA175F1
:1019C70090FF00121E0C00121D6D4004EF20E0EF87
:1019D700A203B34004EF30E003D38001C392043085
:1019E700040302195D121E1300781DE6244DF582CB
:1019F700E4340C121DE280BB9016907401F0122E95
:101A070052781FE66450702B18E670277822F67F0D
:101A17000112292F3004037F01227F0112292F3061
:101A270004037F01227F6012292F3004037F0122E4
:051A37007FFF227F018A
:0B1A3C00227E0212002A781FA607225B
:102BDD007808E6900C49121D5FEDD3940040101D4E
:102BED00744D2DF582E4340CF583E02EFE80EAEE73
:0E2BFD00F404FE744D2FF582E4340C121DEB2F
:012C0B0022A6
:10269000901690E060607810E67034122BDD781CA4
:1026A000121DAC60107A0C7948121E2D1229D678B2
:1026B0001CA6078013781C121D947A0C7948121DF1
:1026C00053781CE690157DF0122DA5121D882278F6
:1026D00018E66022121DC3401D121E1A4014E49019
:1026E0001690F0122E1F780806E670027601E47844
:0626F00013F6E47810F679
:0126F60022C1
:101A47007F58121B3D20040E781FE6FE70037F01AE
:101A570022EE6401601FC202120B3AEF4E70F7903C
:101A67000D527450F0900D507401F0901691F012D1
:101A77002E527F01227F8A7E0212002A781EA60735
:101A87002004D37F8A121B3D2004CB781FE6FEB4C7
:101A9700C0037F0022781EE6FD70037F0122121D1E
:101AA700D950B3900D52EEF0781EE616900D50F017
:101AB700E418F6791DE7C3781E96503C121DA175F0
:101AC70090FF00121E0C00121D6D4004EF20E0EF86
:101AD700A203B34004EF30E003D38001C392043084
:101AE7000403021A5D121E1300781DE62453F582C3
:101AF700E4340D121DE280BB9016917401F0122E92
:101B070052781FE66450702B18E670277822F67F0C
:101B17000112292F3004037F01227F0112292F3060
:101B270004037F01227F6012292F3004037F0122E3
:051B37007FFF227F0189
:0B1B3C00227E0212002A781FA607225A
:102C0C007808E6900D4F121D5FEDD3940040101D17
:102C1C0074532DF582E4340DF583E02EFE80EAEE3C
:0E2C2C00F404FE74532FF582E4340D121DEBF8
:012C3A002277
:1026F700901691E060607810E67034122C0C781C0C
:10270700121DAC60107A0D794E121E2D1229D67843
:102717001CA6078013781C121D947A0D794E121D82
:1027270053781CE690157DF0122DA5121D8822788E
:1027370018E66022121DC3401D121E1A4014E490B1
:102747001691F0122E1F780806E670027601E478DB
:0627570013F6E47810F611
:01275D002259
:101B47007F58121C3D20040E781FE6FE70037F01AC
:101B570022EE6401601FC202120B3AEF4E70F7903B
:101B67000E587450F0900E567401F0901692F012C1
:101B77002E527F01227F8A7E0212002A781EA60734
:101B87002004D37F8A121C3D2004CB781FE6FEB4C5
:101B9700C0037F0022781EE6FD70037F0122121D1D
:101BA700D950B3900E58EEF0781EE616900E56F008
:101BB700E418F6791DE7C3781E96503C121DA175EF
:101BC70090FF00121E0C00121D6D4004EF20E0EF85
:101BD700A203B34004EF30E003D38001C392043083
:101BE7000403021B5D121E1300781DE62459F582BB
:101BF700E4340E121DE280BB9016927401F0122E8F
:101C070052781FE66450702B18E670277822F67F0B
:101C17000112292F3004037F01227F0112292F305F
:101C270004037F01227F6012292F3004037F0122E2
:051C37007FFF227F0188
:0B1C3C00227E0212002A781FA6072259
:102C3B007808E6900E55121D5FEDD3940040101DE1
:102C4B0074592DF582E4340EF583E02EFE80EAEE06
:0E2C5B00F404FE74592FF582E4340E121DEBC2
:012C69002248
:10275E00901692E060607810E67034122C3B781C74
:10276E00121DAC60107A0E7954121E391229D678C9
:10277E001CA6078013781C121D947A0E7954121D14
:10278E0053781CE690157DF0122DA5121D88227827
:10279E0018E66022121DC3401D121E1A4014E4904A
:1027AE001692F0122E1F780806E670027601E47873
:0627BE0013F6E47810F6AA
:0127C40022F2
:101C47007F58121D3D20040E781FE6FE70037F01AA
:101C570022EE6401601FC202120B3AEF4E70F7903A
:101C67000F5E7450F0900F5C7401F0901693F012B1
:101C77002E527F01227F8A7E0212002A781EA60733
:101C87002004D37F8A121D3D2004CB781FE6FEB4C3
:101C9700C0037F0022781EE6FD70037F0122121D1C
:101CA700D950B3900F5EEEF0781EE616900F5CF0F9
:101CB700E418F6791DE7C3781E96503C121DA175EE
:101CC70090FF00121E0C00121D6D4004EF20E0EF84
:101CD700A203B34004EF30E003D38001C392043082
:101CE7000403021C5D121E1300781DE6245FF582B3
:101CF700E4340F121DE280BB9016937401F0122E8C
:101D070052781FE66450702B18E670277822F67F0A
:101D17000112292F3004037F01227F0112292F305E
:101D270004037F01227F6012292F3004037F0122E1
:051D37007FFF227F0187
:0B1D3C00227E0212002A781FA6072258
:102C6A007808E6900F5B121D5FEDD3940040101DAB
:102C7A00745F2DF582E4340FF583E02EFE80EAEED0
:0E2C8A00F404FE745F2FF582E4340F121DEB8C
:012C98002219
:1027C500901693E060607810E67034122C6A781CDD
:1027D500121DAC60107A0F795A121E391229D6785B
:1027E5001CA6078013781C121D947A0F795A121DA6
:1027F50053781CE690157DF0122DA5121D882278C0
:1028050018E66022121DC3401D121E1A4014E490E2
:102815001693F0122E1F780806E670027601E4780A
:0628250013F6E47810F642
:01282B00228A
:08290A0041147906411478150F
:100C4300E4780FF67809F69014787E157F7DE0FD41
:100C530022E02405FFE433FE7809E6C39FEE6480B7
:100C6300F874809822A3E0FBA3E475F001120B242F
:100C7300A9F0FA120AE32FFF22901479E09015806D
:100C8300F0E490157EF090157D04F022E4780FF6E1
:100C93007809F6227E147F7A7809E6FD22AE90D297
:100CA300A0D37815E6940018E6940022780DE62484
:100CB30084F582E43416F583E4F022FA7B01E02420
:100CC30005C39D9016ADF022F583E0F590C2A2C254
:100CD300A1C2A022FA7B01C374059D9016ADF02238
:100CE300EFF0E0780926F6E6C39405227601780F43
:100CF3007602E4780BF622EFF0E0FF780926F6EFB0
:100D030022E4F6780B06E6D3940A22E0D394007427
:100D13008094812290157DE0FFA3E06F2278147602
:100D23000208768A227E157F7D901479E0FD22D217
:100D3300A2D2A1C2A0227E147F7A7B01227813E67D
:040D4300D39405221E
:101E4500901062E0781DF6901064E0B4B00AE4905A
:101E55001680F0122E30C322901064E024F054E076
:101E650070117822E670087601781D76018004E409
:101E75007822F67F0112292F300402D322781DE63D
:101E8500FF12292F300402D322901064E0FF12299B
:101E95002F300402D322781D16E4FF781DE6FEEFED
:101EA500C39E5039120D207590FF00120D3200129D
:101EB5000CA04004EE20E0EFA203B34004EE30E0B6
:101EC50003D38001C39204300402D32274652FF535
:101ED50082E43410120CCB00D2A00F80BE7822E62B
:0D1EE50064016008E4901680F0122E30C3F6
:011EF20022CD
:10049800780FE624FE606014700302053B240360B5
:1004A800030205DA120D397A107960122D1A7809CB
:1004B800A607E670030205ED901060E0B40105128E
:1004C8000CEF8033901060E0B40602800C9010604E
:1004D800E0B415BC120D4040187810E6B4070E12AF
:1004E8000CAF122E1F780806E670027601E4781326
:1004F800F6E47810F68099120C972460F9E4341029
:10050800120CD712296A9016A4120CE350030205A4
:10051800DA901063E0F4FF901062E06F6006120C4E
:100528008F0205DA780F7603901062120D0E4003E1
:100538000205CF120C972460F9E43410901062126F
:100548000CBE12296A9016A4120CFA6004E4780B07
:10055800F6901062120C544079901062E0049016E4
:10056800A4F07A107964A37401F0A37410F0A37452
:1005780064F0E4FF9016A4E0FE14F0EE6005120C9F
:100588006880F1EF7041122E7D503C120D17600B00
:10059800901479120C4D122D628003120C7C122DCE
:1005A800A5901061E0600CE07812667006120C8F5E
:1005B800020498901061E07812F69016807401F0A9
:1005C800122E5D120C8F22120C4A122D62122DA5CA
:1005D80080DB7819E6600E120D044009120C4312F4
:0505E8002D62122DA59B
:0105ED0022EB
:101EF300901168E0781DF690116AE0B4B00AE4909E
:101F03001681F0122E30C32290116AE024F054E0BF
:101F130070117822E670087601781D76018004E45A
:101F23007822F67F0112292F300402D322781DE68E
:101F3300FF12292F300402D32290116AE0FF1229E5
:101F43002F300402D322781D16E4FF781DE6FEEF3E
:101F5300C39E5039120D207590FF00120D320012EE
:101F63000CA04004EE20E0EFA203B34004EE30E007
:101F730003D38001C39204300402D322746B2FF580
:101F830082E43411120CCB00D2A00F80BE7822E67B
:0D1F930064016008E4901681F0122E30C346
:011FA000221E
:10089A00780FE624FE606014700302093D240360A9
:1008AA00030209D9120D397A117966122D1A7809BB
:1008BA00A607E670030209EC901166E0B40105127E
:1008CA000CEF8033901166E0B40602800C9011663A
:1008DA00E0B415BC120D4040187810E6B4070E12A9
:1008EA000CAF122E1F780806E670027601E4781320
:1008FA00F6E47810F68099120C972466F9E434111C
:10090A00120CD712296A9016A4120CE3500302099A
:10091A00D9901169E0F4FF901168E06F6006120C3B
:10092A008F0209D9780F7603901168120D0E4003D1
:10093A000209CE120C972466F9E434119011681258
:10094A000CBE12296A9016A4120CFA6004E4780B01
:10095A00F6901168120C544076901168E0049016D3
:10096A00A4F07A11796AA37401F0A37411F0A37444
:10097A006AF0E4FF9016A4E0FE14F0EE6005120C93
:10098A006880F1EF703E122E7D5039120D17600803
:10099A00120D28122D628003120C7C122DA59011C3
:1009AA0067E0600CE07812667006120C8F02089AF3
:1009BA00901167E07812F69016817401F0122E5D9C
:1009CA00120C8F22120C4A122D62122DA580DB788E
:1009DA0019E6600E120D044009120C43122D621220
:0209EA002DA539
:0109EC0022E8
:101FA10090126EE0781DF6901270E0B4B00AE490E1
:101FB1001682F0122E30C322901270E024F054E009
:101FC10070117822E670087601781D76018004E4AC
:101FD1007822F67F0112292F300402D322781DE6E0
:101FE100FF12292F300402D322901270E0FF122930
:101FF1002F300402D322781D16E4FF781DE6FEEF90
:10200100C39E5039120D207590FF00120D3200123F
:102011000CA04004EE20E0EFA203B34004EE30E058
:1020210003D38001C39204300402D32274712FF5CB
:1020310082E43412120CCB00D2A00F80BE7822E6CB
:0D20410064016008E4901682F0122E30C396
:01204E00226F
:1005EE00780FE624FE606014700302069124036007
:1005FE0003020730120D397A12796C122D1A78090E
:10060E00A607E6700302074390126CE0B4010512D0
:10061E000CEF803390126CE0B40602800C90126CDA
:10062E00E0B415BC120D4040187810E6B4070E1257
:10063E000CAF122E1F780806E670027601E47813CE
:10064E00F6E47810F68099120C97246CF9E43412C3
:10065E00120CD712296A9016A4120CE3500302074B
:10066E003090126FE0F4FF90126EE06F6006120C85
:10067E008F020730780F760390126E120D0E400324
:10068E00020725120C97246CF9E43412FA7B0190C0
:10069E00126E120CC112296A9016A4120CFA600482
:1006AE00E4780BF690126E120C54407690126EE0B7
:1006BE00049016A4F07A127970A37401F0A3741248
:1006CE00F0A37470F0E4FF9016A4E0FE14F0EE6058
:1006DE0005120C6880F1EF703E122E7D5039120D0E
:1006EE00176008120D28122D628003120C7C122D39
:1006FE00A590126DE0600CE07812667006120C8FF9
:10070E000205EE90126DE07812F69016827401F0EA
:10071E00122E5D120C8F22120C4A122D62122DA572
:10072E0080DB7819E6600E120D044009120C43129C
:05073E002D62122DA543
:010743002293
:10204F00901374E0781DF6901376E0B4B00AE49024
:10205F001683F0122E30C322901376E024F054E052
:10206F0070117822E670087601781D76018004E4FD
:10207F007822F67F0112292F300402D322781DE631
:10208F00FF12292F300402D322901376E0FF12297A
:10209F002F300402D322781D16E4FF781DE6FEEFE1
:1020AF00C39E5039120D207590FF00120D32001291
:1020BF000CA04004EE20E0EFA203B34004EE30E0AA
:1020CF0003D38001C39204300402D32274772FF517
:1020DF0082E43413120CCB00D2A00F80BE7822E61C
:0D20EF0064016008E4901683F0122E30C3E7
:0120FC0022C1
:10074400780FE624FE60601470030207E724036058
:1007540003020886120D397A137972122D1A780958
:10076400A607E67003020899901372E0B40105121B
:100774000CEF8033901372E0B40602800C90137275
:10078400E0B415BC120D4040187810E6B4070E1200
:100794000CAF122E1F780806E670027601E4781377
:1007A400F6E47810F68099120C972472F9E4341365
:1007B400120CD712296A9016A4120CE350030208F3
:1007C40086901375E0F4FF901374E06F6006120CCA
:1007D4008F020886780F7603901374120D0E40036F
:1007E40002087B120C972472F9E43413FA7B01900B
:1007F4001374120CC112296A9016A4120CFA600424
:10080400E4780BF6901374120C544076901374E051
:10081400049016A4F07A137976A37401F0A37413E8
:10082400F0A37476F0E4FF9016A4E0FE14F0EE60FA
:1008340005120C6880F1EF703E122E7D5039120DB6
:10084400176008120D28122D628003120C7C122DE1
:10085400A5901373E0600CE07812667006120C8F9A
:10086400020744901373E07812F69016837401F033
:10087400122E5D120C8F22120C4A122D62122DA51B
:1008840080DB7819E6600E120D044009120C431245
:050894002D62122DA5EC
:01089900223C
:100080000000000600000001000000340001C20072
:040090004C5053007D
:10291200441694000000104416A000000100441662
:0C292200980000000044169C000000001B
:092EA300C2AF78257632D2AF22CD
:072EB30075A61E75A6E122C1
:04000600C2AF80FE07
:10211A00020329E493A3F8E493A34003F68001F2AF
:10212A0008DFF48029E493A3F85407240CC8C333C6
:10213A00C4540F4420C8834004F456800146F6DF95
:10214A00E4800B01020408102040809028F4E47E09
:10215A00019360BCA3FF543F30E509541FFEE4938A
:10216A00A360010ECF54C025E060A840B8E493A351
:10217A00FAE493A3F8E493A3C8C582C8CAC583CA7C
:10218A00F0A3C8C582C8CAC583CADFE9DEE780BE34
:01292E0000A8
:1009ED00E709F608DFFA8046E709F208DFFA803EEC
:1009FD0088828C83E709F0A3DFFA8032E309F608D9
:100A0D00DFFA8078E309F208DFFA807088828C8340
:100A1D00E309F0A3DFFA806489828A83E0A3F608F4
:100A2D00DFFA805889828A83E0A3F208DFFA804CCE
:100A3D0080D280FA80C680D4806980F280338010A5
:100A4D0080A680EA809A80A880DA80E280CA80330E
:100A5D0089828A83ECFAE493A3C8C582C8CCC58386
:100A6D00CCF0A3C8C582C8CCC583CCDFE9DEE78056
:100A7D000D89828A83E493A3F608DFF9ECFAA9F0D5
:100A8D00EDFB2289828A83ECFAE0A3C8C582C8CC2B
:100A9D00C583CCF0A3C8C582C8CCC583CCDFEADE44
:100AAD00E880DB89828A83E493A3F208DFF980CCA6
:100ABD0088F0EF60010E4E60C388F0ED2402B4049F
:100ACD000050B9F582EB2402B4040050AF23234546
:060ADD008223900A3D7324
:100AE300BB010689828A83E0225002E722BBFE0211
:090AF300E32289828A83E4932244
:100AFC00BB010689828A83F0225002F722BBFE01D9
:020B0C00F322D2
:100B0E00C5F0F8A3E028F0C5F0F8E5821582700272
:060B1E001583E038F0220F
:100B2400A3F8E0C5F025F0F0E58215827002158384
:060B3400E0C838F0E822E1
:00000001FF
